:105D8A00011900002D0101010200000301FA0400BB
:105D9A00FA0500030A0A5A0B001E0C00FA0D00034A
:105DAA000E00040F0164100096120132130AFA144D
:105DBA00010215000017010A1801FA1905321A0121
:105DCA000A1B01FA1C05321FFFFF20FFFF23011ED9
:105DDA002400642A00FA2B00FA2C50782D003C2E5D
:105DEA0000462F001E3000643250783300003432EF
:105DFA00FA350164360164370150380A643C00649C
:105E0A003E003C3F000040FFFF411450420A5A4303
:105E1A000AC84405324500B44600FA47FFFF480263
:105E2A00024C00FA4EFFFF500808510596520A32FA
:105E3A00530B46540A965601015705465800025913
:105E4A000A465A32FA5B010A5C0A325E000A5F00AD
:105E5A00FE61FFFF64FFFF66000267FFFF6A0A3CFC
:105E6A006B00006C3296730000740000780132797E
:105E7A0001327EFFFF81FFFF84FFFF8500AF8600AE
:105E8A00018700FA89010A8A00009900009D0A9692
:105E9A009E00019FFFFFA0FFFFFAFAFA0065006F5C
:105EAA0000790083008D009700A100AC00B600C005
:105EBA0000CA00D400DE00E800F200580060006862
:105ECA0000700078008000880090009800A000A868
:105EDA0000B000B800C100C800D000D800DF00E65A
:105EEA0000EE00F600410047004D00530059005FE4
:105EFA000065006C00710077007D00830089008FC7
:105F0A000095009B00A200A700AC00B200B900C037
:105F1A0000C500CA00D200D500DD00E100E700EFAD
:103A39009007A9E0FEA3E0FF905D8C126063E49318
:103A4900F599905D8AE493FC740193FDEFB5050740
:103A5900EEB504037576009007A912604A22AE35C7
:103A6900AF3674B48E048F05FF12602C8C378D38F5
:103A7900AE35AF3674B48E048F05FF1260578C359E
:103A89008D36E5364535601374B4C39536FFE49534
:103A990035FE8E358F367837126090E54FA837B8E6
:103AA9000015D395384010E54FC39538FFE4953795
:103AB900FE8E378F388010E54F2402C39538FFE416
:103AC9009537FE8E378F3822900079E0B40104C211
:103AD900108002D21090007AE0B40104C211800271
:103AE900D2119000B7E075F0C3A4FFAEF0740A8E4E
:103AF900048F05FF12602C90079FECF0A3EDF07482
:103B0900038C068D0712603C740112003990079DE1
:103B1900EEF0A3EFF0740312603C740112003990C7
:103B2900000DEEF0A3EFF09000C3E060139000C326
:103B3900E0F5F0741684FD7C00ED9007B1F0800685
:103B490074649007B1F09000B9E090005AF09001C8
:103B590003E0900044F0900092E0900046F090005D
:103B6900BBE0900047F0900067E0900048F09000BB
:103B7900EDE090004DF0900151E090004EF0900181
:103B890052E090004FF0900153E0900050F0A227CE
:103B9900B34016900151E0700C900152E07006900C
:103BA9000153E060028002C2279000A0E0B4010541
:103BB900753B00801F7E017F00900075E012603C1C
:103BC9009000B8E08E048F05FF12602C740AFF1272
:103BD900602C8D3B9000C1E075F0C3A4FFAEF0747A
:103BE9000A8E048F05FF12602C9007A3ECF0A3ED59
:103BF900F0900065E0D3945940067459900065F03F
:103C0900740290005DF0900065E0245A90005EF027
:103C190074E3900059F09000A2E0B40B0874E390AB
:103C29000059F0805A9000A2E0B419129000B8E04F
:103C3900905E9112008CE493900059F080419000BD
:103C4900A2E0B41E129000B8E0905EAF12008CE4BE
:103C590093900059F080289000A2E0B428129000B7
:103C6900B8E0905ED912008CE493900059F0800F6F
:103C79009000A2E0B44608900099E0900059F090B5
:103C89000035E0C39405500D9000BDE0B402067400
:103C9900019000BDF09000D2E0FE9000A0E06E60BF
:103CA9000A9000A0E09000D2F0D226900064E0FED5
:103CB9009000B5E0B5063F90005FE0FE90009FE000
:103CC900B50633900061E0FE9000BDE0B50627908F
:103CD9000060E0FE9000CBE0B5061B900063E0FEBB
:103CE900900072E0B5060F900062E0FE9000ADE032
:103CF9006E7003023E21900035E0C39404500874AD
:103D0900029000EEF08028900035E0C3940450083A
:103D190074069000EEF0801790005DE0C3940350A4
:103D290008740A9000EEF0800674069000EEF09098
:103D39000035E0D3940440099000BDE0D3940150CC
:103D490002800874179000F0F0800674009000F06B
:103D5900F090009FE06008741A900086F0800C745F
:103D690000900086F07400900087F090009FE0B406
:103D790002087419900087F080067400900087F09B
:103D89009000CBE0701474069006C7F07405900695
:103D9900CBF074049006CFF0802474009006C7F02D
:103DA90074009006C8F074009006CBF07400900679
:103DB900CCF074009006CFF074009006D0F0D226B3
:103DC90090009FE090005FF09000CBE0900060F0E1
:103DD9009000BDE0900061F09000ADE0900062F0CD
:103DE900900072E0900063F09000B5E0900064F0FC
:103DF900900072E0900045F09000ADE0900049F02D
:103E09009000CBE090004AF090009FE090004BF0CA
:103E19009000BDE090004CF09000D5E0B4011790FF
:103E2900001B740FF0A374FFF090001DE4F0A3F0E1
:103E390074029000D5F09000D5E0B4034190001DC4
:103E4900E0FEA3E0FF90001BE0FCA3E0FD12608808
:103E5900741012603C7408120039EF900056F0EFAC
:103E6900700674FF900056F074009000D5F0900031
:103E79001CE0900057F090001BE0900058F0752866
:103E89000122C293C294C291C292C287C290E5B57F
:103E990054EFF5B5E5B554DFF5B5C296C295C2A0A4
:103EA900C297C2A2C2A1E5B554BFF5B5E5B5547F25
:103EB900F5B5E5B554FBF5B5C2127539469000AFB5
:103EC900E070057548028003754803752C00752B51
:103ED9000090000874FFF0A374DCF0C218C21A74D1
:103EE900C8900027F074C8900029F0752A00752938
:103EF90000C20D756F00E54AB40903754A00753EA5
:103F090000900011E4F0A3F0754B10C215C216C25F
:103F19001790079FE0FEA3E0FF740312603C740151
:103F290012003990079DEEF0A3EFF0C202C221758D
:103F39002E00752D00C228753000752F0090007174
:103F4900E075F032A4FDACF0900019ECF0A3EDF0AF
:103F5900C238754E0090001F74FFF0A374DCF09016
:103F6900002374FFF0A374DCF0900021E4F0A3F0C7
:103F7900A22CB39205A22DB39206A22EB39207A248
:103F89002FB39208A230B39209A231B3920AA23296
:103F9900B3920BA233B3920C2275A71085F94F8502
:103FA900FA507E017F00E55012603CE54F2FFF502B
:103FB900010E8E358F36AC37AD38EF2DFDEE3CFC5A
:103FC9008C378D38D293D294D291D292E538F5FBC1
:103FD900E537F5FCE538F5E9E537F5EAE538F5EBD8
:103FE900E537F5ECE538F5EDE537F5EE75A700228F
:103FF90085F94F85FA507E017F00E55012603CE556
:104009004F2FFF50010E8E358F367E017F7690003F
:10401900EAE012603CAC35AD36ED2FFFEC3EFE8E8A
:10402900378F38E538F5E9E537F5EA90005AE4F0D5
:104039007412900032F022A215B3B35006E5396428
:10404900016002804DA201B35006A200B3B3400241
:10405900803C75A71085F94F85FA507E017F00E5F0
:104069005012603CE54F2FFF50010E8E358F369070
:10407900000FE0FCA3E0FDEF2DFDEE3CFC8C378D3D
:1040890038E538F5FBE537F5FCD29375A700C2157D
:10409900D216A216B3B35006E53964026002804D08
:1040A900A201B35006A200B3B34002803C75A71029
:1040B90085F94F85FA507E017F00E55012603CE595
:1040C9004F2FFF50010E8E358F3690000FE0FCA365
:1040D900E0FDEF2DFDEE3CFC8C378D38E538F5E938
:1040E900E537F5EAD29475A700D215C216A215B321
:1040F900B35006E53964036002804DA201B350064E
:10410900A200B3B34002803C75A71085F94F85FA28
:10411900507E017F00E55012603CE54F2FFF5001B2
:104129000E8E358F3690000FE0FCA3E0FDEF2DFDDC
:10413900EE3CFC8C378D38E538F5EBE537F5ECD2FC
:104149009175A700C215D216A216B3B35006E53968
:1041590064046002804DA201B35006A200B3B340CB
:1041690002803C75A71085F94F85FA507E017F00C2
:10417900E55012603CE54F2FFF50010E8E358F360A
:1041890090000FE0FCA3E0FDEF2DFDEE3CFC8C3729
:104199008D38E538F5EDE537F5EED29275A700D201
:1041A90015C21622053F22A2D8B34002D221A2D8B5
:1041B900B34002C296A2D9B340089000B9E090007A
:1041C9005AF075D8402285A74D75A710A2D8B340DB
:1041D90002C293A2D9B34002C294A2DAB34002C286
:1041E90091A2DBB34002C29275D840854DA72290B7
:1041F9000047E4936406600280FE74C89007A5F83E
:10420900E4F0E8A3F075B50075840175A70075FFA2
:10421900A090002FE4F075C91075A70F75A1C77597
:10422900A70075D90075CE0C75A70F75F1FE75F24B
:10423900FF75F30775F47875A4BA75A5FF75A60718
:1042490075AE0075AFFF75D48175D5FF75D6FF754D
:10425900D7FF75A70075A20175A14775F80975D82B
:104269000075D90475DA0975D84075A71075D80095
:1042790075D90475DA0975DB0975DC0975DD097508
:10428900D84075A70075E60875E71075BC0175BEBD
:104299000475BD6C75BE0775BDA075BE0875BD01F9
:1042A90075BC0075BB1875BC2075BA0875E88075B2
:1042B900D11375A70F75E10575E20075C740123E68
:1042C9008B759700759780740A12601C7597C0E505
:1042D900975420700280F8758F0275A700D2AF75C8
:1042E900980075A90C75A70F75AB4375ADFB75AC37
:1042F9001E75A71075C91875CA0075CB0075C80455
:1043090075A700758912758E04758C00758A00C2AF
:10431900A9D28C758D00758B00D2ABD28E75EF0644
:1043290075D944C29974C8F5097508001200E97570
:10433900B5001204E974639007A5F8E4F0E8A3F066
:1043490012037574C89007A5F8E4F0E8A3F0746443
:10435900F5097508001200E9900045E0900072F037
:10436900900072E0D39403400C7400900072F074D2
:1043790000900045F0C21E900072E09059B9F828EB
:1043890028738028A2B44002D21E802075A70F7519
:10439900F30F75A700A2A34002D21E800F75A70FC5
:0C43A90075F31775A700A2A44002D21EF5
:0C59B90002438B02438D0243950243A67B
:1043B500A21EB3405F754F08E54FD3940E5020E51C
:1043C5004F9007A5F8E4F0E8A3F01202447464F5F1
:1043D500097508001200E9784F740126F650D97462
:1043E500029000AEF0900045E0900072F0900072EF
:1043F500E09059C5F8282873801674009000D8F00D
:10440500800E74009000BDF0800674009000CAF024
:0C59C5000243FD0243FF02440702440FAE
:10441500D21D805D754F01E54FD394075020E54FC0
:104425009007A5F8E4F0E8A3F01202447464F509D6
:104435007508001200E9784F740126F650D9740109
:104445009000AEF0900045E0900072F0900072E0B0
:104455009059D1F8282873801674009000D8F08000
:0F4465000E74009000BDF0800674009000CAF045
:0C59D10002445C02445E02446602446E24
:10447400C21D900044E0900103F0900045E09000DC
:1044840072F0900046E0900092F0900047E09000B7
:10449400BBF0900048E0900067F0900049E0900085
:1044A400ADF090004AE09000CBF090004BE090001B
:1044B4009FF090004CE09000BDF090004DE0900023
:1044C400EDF090004EE0900151F090004FE090012B
:1044D40052F0900050E0900153F0900151E0700CC4
:1044E400900152E07006900153E060028004C227FC
:1044F4008002D2279000B8E07006740A9000B8F0E9
:10450400900099E0700674E3900099F090009FE0A9
:104514000490005FF09000A0E09000D2F0123AD135
:10452400E5B54401F5B57406900033F074019000CC
:1045340034F07403900036F07405900037F074473B
:10454400900038F07404900039F0740190003AF04F
:10455400740090003FF07400900042F074FF9000EB
:1045640043F0743890013CF0744390013DF0747949
:1045740090013EF0746C90013FF07420900140F083
:10458400744C900141F07461900142F07472900196
:1045940043F07467900144F07465900145F0742011
:1045A400900146F07453900147F0746C900148F008
:1045B400746F900149F0747490014AF09000D4E053
:1045C400900056F090008BE0900057F090008CE043
:1045D400900058F0A2B6B3920EA2B3B3920FA2A465
:1045E400B39223A2B4B39224A2A3B392259000520F
:1045F400E4F0754A00743A900765F074FD9007661C
:10460400F0900053E4F090079FE0FEA3E0FF7403F2
:1046140012603C740112003990079DEEF0A3EFF094
:10462400754901900032E4F0C222753E00C213D2F3
:1046340014C202754C00C22AD203C22BD204C22C6B
:10464400D205C22DD206C22ED207C22FD208C23042
:10465400D209C231D20AC232D20BC233D20CC21F27
:10466400C220C22612009E753A00754600753C00B1
:1046740075403275410075420075430075440075FC
:104684004500900011E4F0A3F0754700D2B2D2A423
:10469400D2B0D2B1D2A3D2A7D2A6D2A5D2B790001B
:1046A40071E0D394FA400674FA900071F07E017FB1
:1046B40000900058E012603C900057E02FFF50013A
:1046C4000E90001BEEF0A3EFF0EFD394FFEE940FE7
:1046D400400790001BE4F0A3F0900056E0700674CD
:1046E400FF900056F09000AEE0D3940240067401AF
:1046F4009000AEF09000AFE070057548028003753D
:1047040048039000B0E0D39401400674009000B0D8
:10471400F09000B6E0C3940A5006740A9000B6F014
:104724009000C0E0700674019000C0F09000C0E0FA
:10473400B4FF0674FE9000C0F09000C7E0D394FE6E
:10474400400674FE9000C7F09000EDE0D394024060
:104754000674019000EDF0900103E0D3940140064B
:104764007401900103F074019000CDF07401900085
:10477400CEF074009000D5F074009000F5F0742928
:104784009006ABF0742A9006AFF074169006B3F05E
:1047940074079006B7F074089006BBF0741B90067B
:1047A400BFF0741C9006C3F0D29C9000A0E0D39498
:1047B40004400674049000A0F0E54BD39410400329
:1047C400754B109006ACE0D3940C40067400900630
:1047D400ACF09006B0E0D3940C400674009006B0A0
:1047E400F09006B4E0D3940C400674009006B4F044
:1047F4009006B8E0D3940C400674009006B8F0908C
:1048040006BCE0D3940C400674009006BCF09006FD
:10481400C0E0D3940C400674009006C0F09006C427
:10482400E0D3940C400674009006C4F09006C8E0EF
:10483400D3940C400674009006C8F09006CCE0D3E4
:10484400940C400674009006CCF09006D0E0D3940B
:104854000C400674009006D0F0D2EC75CF01A298FB
:10486400B34005C298120646E5766006A299B3B332
:1048740040028005C299120C57E57764016005E592
:1048840077B4040280D5C28E7E107F00E53F1260AB
:104894003CE58D75F010A4FDACF0EF2DFDEE3CFC75
:1048A400E58B75F01084FF7E00ED2FFFEC3EFE8E4D
:1048B4002B8F2CD28E900092E060569000131260E1
:1048C4004A900013E0FCA3E0FD900015E0FAA3E099
:1048D400FBEDB5033CECB50238B21CA20DB340139A
:1048E400A21CB34008E5B54404F5B58006E5B5540B
:1048F400FBF5B5900015E0FEA3E0FF900017E0FC87
:10490400A3E0FDEF2DFDEE3CFC900015ECF0A3EDD3
:10491400F090009FE0600990009FE0C39403400280
:10492400806F122D96A20DB35009900052E0C394EB
:104934000740028006900089E0F56EE56E75F0058B
:10494400A4FFAEF09007A7EEF0A3EFF0900076E09E
:10495400C3953C4007E53AC3953B50079007A7E44D
:10496400F0A3F0AE57AF589007A7E0FCA3E0FDEF2B
:10497400D39DEE9C4004C2A1800B900052E0C394EE
:104984000B5002D2A190009FE0B40205A2A1B39201
:10499400A290009FE0B4031C122EB1AE57AF589002
:1049A40007A7E0FCA3E0FDEFD39DEE9C4004D2A159
:1049B4008002C2A1A2B6300E01B35003024E9DA2E2
:1049C400B6300E01B35003024E9DA2B6301001B3AF
:1049D4005003024CEA7549000539E548B40354AE66
:1049E4002BAF2C7401120039900008E0FCA3E0FD09
:1049F40074038F02FF12602CEDC39AEC9E4022AE2A
:104A04002BAF2C74038E048F05FF12602C900008CA
:104A1400E0FEA3E0FF7401120039EFD39DEE9C4049
:104A240005754801800BA228B3400690003274013A
:104A3400F0D228E548B40203754801E5487048AE51
:104A44002BAF2C7401120039900008E0FCA3E0FDA8
:104A540074038F02FF12602CEAC39DEE9C4022AEC9
:104A64002BAF2C74038E048F05FF12602C9000086A
:104A7400E0FEA3E0FF7401120039EDD39FEC9E40E9
:104A8400067402900032F0AE2BAF2C900025E0FCAF
:104A9400A3E0FD12608874038F028E038C068D07D9
:104AA40012603C7401120039EAD39FEB9E400AE580
:104AB400487006A212B3B340028003753901900016
:104AC40008E52BF0A3E52CF0AE2BAF2C74098E0473
:104AD4008F05FF12602C8C2D8D2EAE2BAF2C740104
:104AE4001200398E338F34AC2FAD30AA2BAB2CEDA2
:104AF4002BFBEC3AFA8A2F8B30AC2BAD2CEDD39BED
:104B0400EC9A401190000BE0F9A3E0FEEEC394E8A8
:104B1400E994034002800690000B12604A900092D0
:104B2400E06043900013E0FEA3E0FF900092E08E6B
:104B3400048F05FF12602C74018C068D0712003956
:104B4400900017EEF0A3EFF0900017E0F8A3E090C8
:104B54000015C8F0A3C8F0900013E4F0A3F0C21C41
:104B6400E5B554FBF5B5C28E758D00758B00753FA8
:104B740000752C01752B00D28E900008E0FEA3E096
:104B8400FFEF4E601074011200397C3B7DD0125F40
:104B94002A8E298F2AAE29AF2A7428BE00039F507B
:104BA40010E53E2FFF50010E74011200398E298F3B
:104BB4002A852A3E9000B6E0A829B8000DD3952A8C
:104BC4004008E52A900031F080099000B6E0149086
:104BD4000031F0E5486006752A007529001223D2D9
:104BE400A212B35003024CAAE539D39404400375CE
:104BF4003901A2135003024CA290006BE0B401737C
:104C04009000EDE0B40214120E2690005BE075F003
:104C1400BEA4FFAEF08E378F388056E54275F00A99
:104C240084FF7E00900565126063E0F536753500FB
:104C3400AE35AF36900090E012603C74648E048F01
:104C440005FF12602C8C378D38E53890000AF0AEE1
:104C540035AF36900069E012603C74648E048F05B1
:104C6400FF12602C74BE8C068D0712603C8E378F49
:104C7400388017900069E075F0BEA4FFAEF08E375F
:104C84008F38900090E090000AF0E53CC394CC503B
:104C940006E538453770028003123FA2D213E54877
:104CA400B40103754B01E54870379000B2E0D3942A
:104CB40001400D90005AE0A829B80006952A400248
:104CC400801C9000B2E0B40305754B038002C2005F
:104CD40090005AE060067409900032F08003754B2E
:104CE40001A210B3920EA210B330B601B350030266
:104CF4004E9D754901E5B54401F5B5740790005220
:104D0400F0A210920EE539D394484002D2129000DA
:104D140025E52BF0A3E52CF0E54AB40903754A0018
:104D24009000BAE0B40107E545C394144002800939
:104D3400123E8B7413900032F0A22A300301B35058
:104D440017A22AB34008E5B54408F5B58006E5B5D1
:104D540054F7F5B5A22A9203A22B300401B35017DD
:104D6400A22BB34008E5B54402F5B58006E5B55479
:104D7400FDF5B5A22B9204A22C300501B3500FA26D
:104D84002CB34004D2958002C295A22C9205A22D88
:104D9400300601B35017A22DB34008E5B54410F511
:104DA400B58006E5B554EFF5B5A22D9206A22E30D6
:104DB4000701B35017A22EB34008E5B54420F5B55A
:104DC4008006E5B554DFF5B5A22E9207A22F300870
:104DD40001B35017A22FB34008E5B54440F5B580A0
:104DE40006E5B554BFF5B5A22F9208A230300901EB
:104DF400B35017A230B34008E5B54480F5B580063A
:104E0400E5B5547FF5B5A2309209A231300A01B359
:104E1400500FA231B34004D2908002C290A23192CA
:104E24000AA232300B01B3500FA232B34004D2872E
:104E34008002C287A232920BA233300C01B3500F0E
:104E4400A233B34004D2928002C292A233920CE500
:104E540045C394415009740E900032F0123E8B9079
:104E64000039E0FE900035E0C39E4009900035E033
:104E7400D39408400974FB900032F0123E8B9000EA
:104E84003EE0601590003EE0FE900038E06E600960
:104E940074FE900032F0123E8B124040E54B905964
:0C4EA400DDF828287302557C9000A0E087
:0659DD00024EA9024EACCF
:104EB000905A10F8282873121EAE8012121EAE806F
:0E4EC0000D121F388008121FE48003121FE439
:0F5A1000024EB7024EBC024EC1024EC6024ECB32
:104ECE00754B0202557C122110122227A238B340D4
:104EDE000C900094E0F5477410900032F085475F17
:104EEE00900008E0FEA3E0FF90000DE0FCA3E0FDC3
:104EFE00EDD39FEC9E4019740212603C74038E0435
:104F0E008F05FF12602C900000ECF0A3EDF0800FE7
:104F1E0090079DE0F8A3E0900000C8F0A3C8F075DC
:104F2E004B03A2394003754B0A02557C9006ACE048
:104F3E0060031224EA9000EBE0B401149000ECE060
:104F4E00A829B80004952A5007E53AC3953B4002BC
:104F5E0080097415900032F0024FEA9000A0E0D361
:104F6E009402403F900074E02403A829B8000495F1
:104F7E002A5009900076E0D3953C50028008D20169
:104F8E007408900032F0900074E0A829B80005D3A0
:104F9E00952A500B900076E02403C3953C5002C234
:104FAE00018039900074E02403A829B80004952AE2
:104FBE005007E53AC3953B40028008D20174089031
:104FCE000032F0900074E0A829B80005D3952A505D
:104FDE0009E53B240FC3953A5002C2019000BAE096
:104FEE007007E545C3941440028002D201A201402D
:104FFE0005754B04800A754B10900011E4F0A3F078
:10500E00A20DB3405DE54275F00A84FF7E00900567
:10501E0065126063E0C39469501F12240790079DC8
:10502E00E0FEA3E0FF740312603C7401120039909D
:10503E00000DEEF0A3EFF0802990079FE0F8A3E0BB
:10504E0090079DC8F0A3C8F090079DE0FEA3E0FF77
:10505E00740312603C740112003990000DEEF0A33F
:09506E00EFF002557C9000A0E077
:0959E300024ED4024F3A02507347
:10507700905A1FF8282873120F108012120F1080F1
:0E5087000D1210BE80081211708003121170FD
:0F5A1F0002507E02508302508802508D02509236
:105095009006B0E060031225C6754B0502557C12DB
:1050A50012B0754B069006B4E060031226B6900662
:1050B500B8E0600312279202557C90000AE0600672
:1050C500A20DB3B34002801D90000AE02552FFAE49
:1050D5005150010E8E518F52E539D39401500690EF
:1050E500000AE014F01214F6754B079006BCE06058
:1050F5000312286E9006C0E0600312294A02557C0F
:105105009000EDE0B40203120E9E1218F5754B08DF
:105115009006C4E06003122A269006C8E0600312D8
:105125002B0202557C121CB1A215B35005A216B371
:1051350040028006D215D216D217754B109006CCB8
:10514500E06003122BDE9006D0E06003122CBA0259
:10515500557C02557C9000B5E0B4050280030252EF
:10516500DD90005EE0D3955F5003025247AE29AF54
:105175002A740ABE00039F501EAE2DAF2E90005E0E
:10518500E0C3955F12603C740C8E048F05FF1260BE
:105195002C8C318D328020AE2DAF2E740C8E048F69
:1051A50005FF12602C90005EE0C3955F8C068D07AD
:1051B50012603C8E318F32900000E0FEA3E0FFAC20
:1051C50031AD32EDD39FEC9E40288F028E038C06C5
:1051D5008D078B048A05126088900021EEF0A3EFFD
:1051E500F0E54EB40207900021E4F0A3F0754E00FF
:1051F500804EE54E7003754E01900008E0FEA3E079
:10520500FFAC31AD32EF2DFDEE3CFC900000E0FA35
:10521500A3E0FBEDD39BEC9A401FAC31AD32EF2DF3
:10522500FDEE3CFC8C068D078A048B051260889088
:105235000021EEF0A3EFF08007900021E4F0A3F049
:105245008074AE2DAF2E90005EE0F404255F1260F1
:105255003C740C8E048F05FF12602C8C318D3290BE
:105265000000E0FEA3E0FFED2FFFEC3EFE900008FE
:10527500E0FAA3E0FBEBD39FEA9E401C8A068B076E
:10528500126088900000E0FCA3E0FD1260889000A9
:1052950021EEF0A3EFF0801E900021E4F0A3F09042
:1052A5000008E0FEA3E0FFAC31AD3212608890004B
:1052B50000EEF0A3EFF0900000E0FEA3E0FF741312
:1052C50012603C74148E048F05FF12602C90000050
:1052D500ECF0A3EDF002548C90005EE0D3955F50A6
:1052E500030253BFAE29AF2A740ABE00039F501EA6
:1052F500AE2DAF2E90005EE0C3955F12603C740A40
:105305008E048F05FF12602C8C318D328020AE2DDE
:10531500AF2E740A8E048F05FF12602C90005EE09C
:10532500C3955F8C068D0712603C8E318F329000DD
:1053350000E0FEA3E0FFAC31AD32EDD39FEC9E4023
:10534500288F028E038C068D078B048A05126088D0
:10535500900021EEF0A3EFF0E54EB4020790002196
:10536500E4F0A3F0754E00804EE54E7003754E01D6
:10537500900008E0FEA3E0FFAC31AD32EF2DFDEE6D
:105385003CFC900000E0FAA3E0FBEDD39BEC9A40D7
:105395001FAC31AD32EF2DFDEE3CFC8C068D078A3E
:1053A500048B05126088900021EEF0A3EFF08007D2
:1053B500900021E4F0A3F002546DAE29AF2A740ADF
:1053C500BE00039F501FAE2DAF2E90005EE0F4048B
:1053D500255F12603C740A8E048F05FF12602C8CC9
:1053E500318D328021AE2DAF2E740A8E048F05FFCC
:1053F50012602C90005EE0F404255F8C068D071288
:10540500603C8E318F32AE31AF32900000E0FCA3AC
:10541500E0FDEF2DFDEE3CFC900008E0FAA3E0FB7B
:10542500EBD39DEA9C40238F048E058A068B07CD1E
:10543500CCCD126088900000E0FCA3E0FD126088EE
:10544500900021EEF0A3EFF0801E900021E4F0A380
:10545500F0900008E0FEA3E0FFAC31AD32126088A9
:10546500900000EEF0A3EFF0900000E0FEA3E0FF57
:10547500741312603C74148E048F05FF12602C9017
:105485000000ECF0A3EDF0E54EB40149754E02E5E0
:1054950048703685F94F85FA507E017F00E5501238
:1054A500603CE54F2FFF50010E8E358F3690000082
:1054B500E0FCA3E0FDEF2DFDEE3CFC8C378D38E5DF
:1054C50038F5FBE537F5FCD29690001F74FFF0A385
:1054D50074DCF0807C90001FE0FEA3E0FFEFB4DCFD
:1054E5002CEEB4FF28900023E0FCA3E0FDEDB4DC36
:1054F5001AECB4FF16900021E0F8A3E090001FC855
:10550500F0A3C8F0900021E4F0A3F08044E54870D2
:105515003685F94F85FA507E017F00E55012603CD3
:10552500E54F2FFF50010E8E358F36900000E0FCC1
:10553500A3E0FDEF2DFDEE3CFC8C378D38E538F50D
:10554500FBE537F5FCD29690001F74FFF0A374DCE1
:10555500F0E548B40112754800754B1090001F74B2
:10556500FFF0A374DCF08003754B03800A8008808C
:0755750006800480028000A3
:1059EC000250A40250BF02510502512A0251570223
:1059FC00515A025572025574025576025578025569
:045A0C007A02557C49
:10557C00AE2BAF2C90001FE0FCA3E0FDEFD39DEE13
:10558C009C4044E548703685F94F85FA507E017F82
:10559C0000E55012603CE54F2FFF50010E8E358F09
:1055AC0036900000E0FAA3E0FBEF2BFBEE3AFA8A10
:1055BC00378B38E538F5FBE537F5FCD29690001FB4
:1055CC0074FFF0A374DCF0A221B3402E900023747E
:1055DC00FFF0A374DCF0900021E0FEA3E0FFEF4E9F
:1055EC006016900021E0F8A3E090001FC8F0A3C85B
:1055FC00F0900021E4F0A3F0C2219000BDE0B402D1
:10560C00028003025722900054E0D39541506490DD
:10561C000054E0F4042541FE9000C0E08E00F5F04B
:10562C00E884FF7E008F4FEFC39410500CEF854F32
:10563C00F0A4FDACF08D4F8003754FFF900054E04B
:10564C00D3954F400B900054E0C3954FF54C80031D
:10565C00754C009000DBE0D3954C40069000DBE0ED
:10566C00F54C9000DCE0C3954C50069000DCE0F566
:10567C004C8071900054E0C39541FE9000C0E08EC8
:10568C0000F5F0E884FF7E008F4FEFC39410500CB0
:10569C00EF854FF0A4FDACF08D4F8003754FFF8567
:1056AC004F36753500900054E02536FFAE3550016D
:1056BC000E8E358F3674FFBE0009D39F400585369C
:1056CC004C8003754CFF9000DBE0D3954C4006906A
:1056DC0000DBE0F54C9000DCE0C3954C50069000EC
:1056EC00DCE0F54CA20DB3B3500D900055E0FE90EC
:1056FC0000C8E0D39E5002800A7407900032F0C2BA
:10570C0097801375A710E5CDC3954C4004C29780C4
:10571C0002D29775A700E54AC39409500AA2EDB3CB
:10572C004005C2ED123050AE2BAF2C7440C39F74A9
:10573C009C9E400C900053E0C3945A40030259B60F
:10574C00A212B34009123E8B7406900032F0A21ED6
:10575C00B34008E5B54404F5B58006E5B554FBF552
:10576C00B5A214B3500EE53CD394334007E53CC3CB
:10577C0094CC400280419000EDE0B40214120E264D
:10578C0090005BE075F050A4FFAEF08E378F388040
:10579C000F900069E075F050A4FFAEF08E378F3893
:1057AC00E53845376011E5B54401F5B5740790004F
:1057BC0052F0123FA2D214900053E0D39401400750
:1057CC00E53CC3941A40028002C2149006ACE0601F
:1057DC00031224EAA22A300301B35017A22AB340C1
:1057EC0008E5B54408F5B58006E5B554F7F5B5A25E
:1057FC002A92039006B0E060031225C6A22B300457
:10580C0001B35017A22BB34008E5B54402F5B5809F
:10581C0006E5B554FDF5B5A22B92049006B4E060F4
:10582C00031226B6A22C300501B3500FA22CB340A4
:10583C0004D2958002C295A22C92059006B8E06025
:10584C0003122792A22D300601B35017A22DB3409C
:10585C0008E5B54410F5B58006E5B554EFF5B5A2ED
:10586C002D92069006BCE0600312286EA22E300723
:10587C0001B35017A22EB34008E5B54420F5B5800E
:10588C0006E5B554DFF5B5A22E92079006C0E06090
:10589C000312294AA22F300801B35017A22FB3408C
:1058AC0008E5B54440F5B58006E5B554BFF5B5A29D
:1058BC002F92089006C4E06003122A26A230300909
:1058CC0001B35017A230B34008E5B54480F5B5805C
:1058DC0006E5B5547FF5B5A23092099006C8E06094
:1058EC0003122B02A231300A01B3500FA231B34084
:1058FC0004D2908002C290A231920A9006CCE06051
:10590C0003122BDEA232300B01B3500FA232B34084
:10591C0004D2878002C287A232920B9006D0E0603C
:10592C0003122CBAA233300C01B3500FA233B34084
:10593C0004D2928002C292A233920C900053E0C324
:10594C00945A5010E54AB40909900053E004F075DC
:10595C004A00803BE54AB40903754A00752C007572
:10596C002B00758D00758B00753F00900052E0C3C5
:10597C00940B5008900052E004F08006740B9000D9
:10598C0052F0900052E0B40B06E5B554FEF5B5901C
:10599C000053E0D394014007E545C3944140028095
:0D59AC0009740E900032F0123E8B02485F2D
:105A2E000000010001400160018001A001C001E001
:105A3E0002000300039603B603D603F40400050028
:105A4E000512052405360548055A056C057E059098
:105A5E0005A805C005DE0600061406280646066ED5
:105A6E0006AE05CF00FF013F015F017F019F01BF21
:105A7E0001DF01FF02FF039503B503D503F303FF17
:105A8E0004FF05110523053505470559056B057DF1
:105A9E00058F05A705BF05CE05F10613062706459A
:105AAE00066D06AD06ED05DD0FAA0FA50F9F0F9A29
:105ABE000F940F8D0F870F800F780F710F680F6087
:105ACE000F570F4E0F450F3B0F300F250F1A0F0EAE
:105ADE000F020EF50EE80EDB0ECC0EBE0EAE0E9FB6
:105AEE000E8E0E7D0E6C0E5A0E470E340E200E0CC0
:105AFE000DF70DE20DCB0DB50D9D0D850D6D0D54F4
:105B0E000D3A0D200D050CE90CCE0CB10C940C7653
:105B1E000C580C3A0C1B0BFB0BDB0BBB0B9A0B79CB
:105B2E000B570B350B130AF10ACE0AAB0A870A6420
:105B3E000A400A1C09F809D409B0098C09670943FF
:105B4E00091F08FB08D608B2088E086A0846082303
:105B5E0007FF07DC07B9079607730751072F070DD5
:105B6E0006EC06CA06AA068906690649062A060A28
:105B7E0005EC05CD05B0059205750558053C0520CB
:105B8E00050504EA04CF04B5049C0482046904519B
:105B9E0004390422040B03F403DE03C803B2039D8D
:105BAE00038903750361034D033B032803160304A6
:105BBE0002F202E102D102C002B002A00291028200
:105BCE000273026502570249023C022F022202169C
:105BDE00020901FD01F201E601DB01D001C601BBA4
:105BEE0001B101A7019D0194018B01820179017020
:105BFE00016801600158015001480141013901322B
:105C0E00012B0125011E01180111010B010500FFD9
:105C1E0000FA0FA60FA00F990F920F8B0F840F7C17
:105C2E000F740F6B0F620F580F4E0F430F380F2C60
:105C3E000F1F0F120F050EF70EE80ED80EC80EB777
:105C4E000EA50E930E800E6C0E580E420E2C0E15D7
:105C5E000DFD0DE40DCB0DB10D950D790D5D0D3FC7
:105C6E000D200D010CE10CC00C9E0C7C0C590C355A
:105C7E000C100BEA0BC40B9E0B760B4F0B260AFD7A
:105C8E000AD40AAA0A800A550A2A09FF09D409A8C1
:105C9E00097C0950092508F908CD08A10875084A9C
:105CAE00081E07F307C8079D07730749072006F765
:105CBE0006CE06A6067E06570630060A05E405BF82
:105CCE00059B057705540532051004EF04CE04AE8E
:105CDE00048F047104530435041903FD03E203C752
:105CEE0003AD0394037B0363034B0334031E0308CA
:105CFE0002F302DE02CA02B602A30291027F026D15
:105D0E00025C024C023C022C021D020E020001F249
:105D1E0001E401D701CA01BE01B101A6019A018FAA
:105D2E000185017A01700166015D0153014A01414D
:105D3E00013901310129012101190112010B01045F
:105D4E0000FD00F700F000EA00E400DE00D900D309
:105D5E0000CE00C900C400BF00BA00B500B100AD4E
:105D6E0000A800A400A0009C009900950091008E50
:0C5D7E00008A008700840081007E007B0A
:10009E007570009007A9E4F0A3F0755A0075590029
:1000AE00757600757700C235D23674FE9007ABF8C0
:1000BE00E4F0E8A3F074FE9007ADF8E4F0E8A3F0E6
:1000CE0074FE9007B7F0745A9007B8F0745A900700
:1000DE00B9F0D237C229C239C23422750B00750A63
:1000EE0000AE0AAF0BAC08AD09EDC39FEC9E4016F7
:1000FE0074FF12601C75CF01780B740126F6500444
:10010E0018E436F650DB2290002FE0B4AA1C9007BC
:10011E0065E0B43C159007A5E0FEA3E0FFEF4E604E
:10012E0009741EBE0004D39F5003020243753800AB
:10013E0075370075F8099007A5E0FEA3E0FF740778
:10014E006F4E6006740E6F4E7006743A900765F02F
:10015E009007A5E0FEA3E0FF7408BE001ED39F40EB
:10016E001A7E017F089007A5E0FCA3E0FD1DBDFFF0
:10017E00011C1200038E358F36801F9007A5E0FEFE
:10018E00A3E0FF74081260808F048E057E017F0845
:10019E00CDCCCD1200038E358F36AE37AF38740C02
:1001AE00D39F74019E500302023EA2F9B3407EE536
:1001BE00384537700375A382AE37AF3874016F4E72
:1001CE00700375A300AE37AF3874026F4E700D908A
:1001DE0007A6E075F002A4FDACF08DA3AE37AF38E4
:1001EE0074036F4E700375A300AE37AF387403BE41
:1001FE0000039F5013AC35AD36ED2FFFEC3EFE9055
:10020E000061126063E0F5A3AE37AF38EFB40B09AF
:10021E00EEB40105741412601CAE37AF38EFB40B98
:10022E0007EEB4010375F80D78371260900201A83D
:10023E0090002FE4F02275380075370075F809909C
:10024E0007A5E0FEA3E0FF7408BE001ED39F401A70
:10025E007E017F089007A5E0FCA3E0FD1DBDFF0118
:10026E001C1200038E358F36801F9007A5E0FEA36B
:10027E00E0FF74081260808F048E057E017F08CD2A
:10028E00CCCD1200038E358F36AE37AF387411D306
:10029E009F74019E5003020374A2F9B3500302032C
:1002AE0071E5384537700375A3D2AE37AF38740198
:1002BE006F4E700375A300AE37AF3874026F4E7079
:1002CE000D9007A6E075F002A4FDACF08DA3AE373D
:1002DE00AF3874036F4E700375A300AE37AF38742A
:1002EE00046F4E700375A300AE37AF3874056F4EB2
:1002FE00700375A300AE37AF3874066F4E7003757A
:10030E00A300AE37AF3874076F4E700375A300AEFF
:10031E0037AF3874086F4E700375A300AE37AF3821
:10032E007408BE00039F5016AC35AD36ED2FFFECB2
:10033E003EFE90005C126063E5A3F075A300AE373D
:10034E00AF38EFB41009EEB40105741412601CAE90
:10035E0037AF38EFB41007EEB4010375F80D7837E8
:10036E001260900202972275380075370075F809F1
:10037E00AE37AF387417BE0004D39F500302044D3E
:10038E00A2F9B3500302044AE5384537700375A34A
:10039E00D2AE37AF3874016F4E700375A300AE370F
:1003AE00AF3874026F4E700D9007A6E075F002A480
:1003BE00FDACF08DA3AE37AF3874036F4E7003757E
:1003CE00A300AE37AF3874046F4E700375A300AE42
:1003DE0037AF3874056F4E700375A300AE37AF3864
:1003EE0074066F4E700375A300AE37AF3874076F87
:1003FE004E700375A300AE37AF3874086F4E70039E
:10040E0075A300AE37AF387408BE00039F500C9032
:10041E00003B126063E5A3F075A300AE37AF3874EE
:10042E00166F4E7005741412601CAE37AF3874160A
:10043E006F4E700375F80D783712609002037E22AE
:10044E0090002FE0B4AB0280030204E8753800750B
:10045E00370075F809AE37AF387412BE007CD39FE3
:10046E004078A2F9B34070E5384537700375A38222
:10047E00AE37AF3874016F4E700375A300AE37AF51
:10048E003874026F4E700D9007A6E075F002A4FD51
:10049E00ACF08DA3AE37AF3874036F4E700375A3F7
:1004AE0000AE37AF387403BE00039F500990004072
:1004BE00126063E0F5A3AE37AF3874116F4E70055E
:1004CE00741412601CAE37AF3874116F4E70037512
:1004DE00F80D7837126090020463229007B4E4F0AE
:1004EE0074649007A5F8E4F0E8A3F012037574C8DD
:1004FE009007A5F8E4F0E8A3F074FF90003BF074C9
:10050E00FF90003CF074FF90003DF07400900035B9
:10051E00F074FF90003EF07400900040F074019073
:10052E000041F0900047E0B4371A900044E090008C
:10053E003BF0900045E090003CF0900046E09000CB
:10054E003DF080469007B47401F074659007A5F8ED
:10055E00E4F0E8A3F012037574C89007A5F8E4F070
:10056E00E8A3F0900047E0B4371A900044E0900002
:10057E003BF0900045E090003CF0900046E090008B
:10058E003DF0800674029007B4F09007B5E4F07465
:10059E00669007A5F8E4F0E8A3F012037574C8900E
:1005AE0007A5F8E4F0E8A3F0900046E0B437129007
:1005BE000044E0900035F0900045E090003EF08061
:1005CE00769007B57401F074679007A5F8E4F0E82B
:1005DE00A3F012037574C89007A5F8E4F0E8A3F031
:1005EE00900046E0B43712900044E0900035F09051
:1005FE000045E090003EF0803E74029007B5F07426
:10060E00689007A5F8E4F0E8A3F012037574C8909B
:10061E0007A5F8E4F0E8A3F0900046E0B437129096
:10062E000044E0900035F0900045E090003EF080F0
:10063E000674039007B5F022E57764046006E59929
:10064E0064FF60028031A2354004D2358027E57701
:10065E00600874E62577900032F0E576600874F055
:10066E002576900032F0E577B4010280FE757700B2
:10067E00757600C2358002C235E57790384AF82883
:10068E002873757700E599B4FF03757601E599B483
:10069E00FE03757602E599B4FD03757603E599B40C
:1006AE00FC03757604E599B4FA03757605E599B4FD
:1006BE00FB06757701123E8BE599B4F90675770442
:1006CE00123E8BE599D394E54007E599C394F0402B
:1006DE000280168599787577027E017F00E578C3D2
:1006EE0094E612603C8E5B8F5C9007A9E4F0A3F059
:1006FE00E599D394C44007E599C394E64002802857
:10070E0085997875770374E5C39578F55C755B000C
:10071E00AE5BAF5C905A2E12600BE493F8740193AB
:10072E009007A9C8F0A3C8F0D299020C56900044C5
:10073E00E07005A227B3400280429007A9E0FEA315
:10074E00E0FF74FFBE00039F5009EFC39446EE9482
:10075E000640119007A9E0FEA3E0FFEFD3946DEEE3
:10076E00940640139007A9E0FEA3E0FF90006512E7
:10077E006063E599F0800385995080119007A9E098
:10078E00FEA3E0FF900065126063E599F09007A963
:10079E0012604A9007A9E0FEA3E0FFEFB40106EE57
:1007AE00B4070280030209FD900765E0B43C0280A5
:1007BE00030209FDA22750030208E8C29C900044E0
:1007CE00E0900103F0900045E0900072F09000463A
:1007DE00E0900092F0900047E09000BBF09000484F
:1007EE00E0900067F0900049E09000ADF090004A74
:1007FE00E09000CBF090004BE090009FF090004C0A
:10080E00E09000BDF090004DE09000EDF090004EB5
:10081E00E0900151F090004FE0900152F0900050A6
:10082E00E0900153F0123AD1900056E09000D4F0CF
:10083E00900057E090008BF0900058E090008CF004
:10084E0074639007A5F8E4F0E8A3F074AB90002F62
:10085E00F012044E90002FE4F07464F50975080050
:10086E001200E9A21D4039754F01E54FD394075090
:10087E002DE54F9007A5F8E4F0E8A3F074AA9000D8
:10088E002FF0120115E54FC39407500A7464F50951
:10089E007508001200E9784F740126F650CC8037A7
:1008AE00754F08E54FD3940E502DE54F9007A5F8E0
:1008BE00E4F0E8A3F074AA90002FF0120115E54FB2
:1008CE00C3940E500A7464F5097508001200E97895
:1008DE004F740126F650CC0209E7C29C900103E04A
:1008EE00900044F0900072E0900045F0900092E08D
:1008FE00900046F09000BBE0900047F0900067E05B
:10090E00900048F09000ADE0900049F09000CBE0F0
:10091E0090004AF090009FE090004BF09000BDE0F8
:10092E0090004CF09000EDE090004DF074009000BF
:10093E004EF0740090004FF07400900050F074630D
:10094E009007A5F8E4F0E8A3F074AB90002FF01236
:10095E00044E90002FE4F07464F50975080012003F
:10096E00E9754F01E54FD394075026E54F9007A543
:10097E00F8E4F0E8A3F074AA90002FF012011574B9
:10098E0064F5097508001200E9784F740126F650D7
:10099E00D3D29C7599FB743C900765F0754F08E5B2
:1009AE004FD3940E5026E54F9007A5F8E4F0E8A338
:1009BE00F074AA90002FF01201157464F5097508F1
:1009CE00001200E9784F740126F650D374C89007D0
:1009DE00A5F8E4F0E8A3F080FE74C89007A5F8E44B
:1009EE00F0E8A3F0D29C7577007576007599FB023E
:1009FE000C569007A9E0FEA3E0FFEF4E7006859916
:100A0E005A7559009007A9E0FEA3E0FF74016F4EDE
:100A1E00701BAC59AD5AAA5BAB5CED2BFBEC3AFAF2
:100A2E008A068B07900065126063E599F09007A91E
:100A3E0012604A9007A9E0FEA3E0FF74026F4E70A9
:100A4E0021AC59AD5A74566D4C7006E57864E6606B
:100A5E00028003123E8B123AD18578997577007514
:100A6E007600020C569007A9E0FEA3E0FF90006509
:100A7E00126063E599F09007A912604A9007A9E009
:100A8E00FEA3E0FFAC5BAD5C8F028E038C068D0780
:100A9E00905A7212600BE493F9740193FEEAD39E9E
:100AAE00EB994009857899757700757600020C569A
:100ABE009007A9E0FEA3E0FF900065126063E59940
:100ACE00F09007A912604A9007A9E0FEA3E0FFEF9D
:100ADE00B40006EEB401028003020C5690003DE015
:100AEE00D394C7400B90003DE0C394C8F579801AAB
:100AFE0090003DE0D39463400B90003DE0C39464BE
:100B0E00F579800690003DE0F579E57975F002A45F
:100B1E00FFAEF08F4FEF90006512606EEFFCE0FDC0
:100B2E00EC90006812606EEDFCE0FDEC2DB57902E4
:100B3E008003020C470FEF90006512606EE54FFFC9
:100B4E00E0FCEF90006912606EECFFE0FCEFC39CDE
:100B5E00B579028003020C47E54F90006712606E74
:100B6E00E54FFFE0FCEF90006A12606EECFFE0FCD8
:100B7E00EF2CB579028003020C47E54F90006B1203
:100B8E00606EE0C39579900044F0E54F90006C12D2
:100B9E00606EE0C39579900045F0E54F90006D12C0
:100BAE00606EE0C39579900046F07400900047F0B7
:100BBE0074FF900048F0E54F90006F12606EE0C336
:100BCE009579900049F0E54F90007012606EE0C389
:100BDE00957990004AF0E54F90007112606EE0C377
:100BEE00957990004BF0E54F90006E12606EE0C369
:100BFE0095799007A5F8E4F0E8A3F074AB90002F78
:100C0E00F012044E7464F5097508001200E990079D
:100C1E00A512604A12044E7464F50975080012009C
:100C2E00E99007A512604A12044E7599F97464F59D
:100C3E00097508001200E980FE7599FF7464F509C4
:080C4E007508001200E980FEA8
:0F384A0002069002073B020A00020A73020ABE3E
:100C560022E576903859F8282873020D699007A97D
:100C6600E0FEA3E0FF900033126063E0F599900781
:100C7600A912604A9007A9E0FEA3E0FF74116F4E27
:100C86007003757600020D69854999020D69900712
:100C9600A9E0FEA3E0FF900065126063E0F599EF1E
:100CA600B40107EEB407037576009007A912604AEF
:070CB600020D699007AAE09E
:0F385900020C60020C63020C8E020C94020CB97C
:100CBD00903A0CF8282873852A99020D5E853A9989
:100CCD00020D5E853C99020D5E854099020D5E8593
:100CDD004299807D854399807885449980738545B7
:100CED0099806E900012E0F5998066A236B34007A8
:100CFD007599FAC2368041A226B3400575990F80C9
:100D0D00359007B4E0600A9007B4E024DCF59980D3
:100D1D00169007B5E0600A9007B5E024DEF59980DE
:100D2D0006900032E0F599900032E4F09007B4E4BB
:100D3D00F09007B5E4F0C22680178546998012859C
:100D4D004199800D85479980087599FC80037576CA
:010D5D000095
:103A0C00020CC4020CCA020CD0020CD6020CDC0252
:103A1C000CE1020CE6020CEB020CF0020CF8020DAD
:0D3A2C0047020D4C020D51020D56020D5BBC
:0B0D5E009007A912604A8003123A3986
:03386800020D66E8
:100D690022E5602536FFAE3550010E900065126010
:100D790063E0F561E5602536FFAE3550010E0FBF22
:100D890000010E900065126063E0F562856864E514
:100D990061B562058561608041E562D39561401D59
:100DA900E562C395618563F0A4FFAEF0E5648E0446
:100DB9008F05FF12602CED2561F560801DE561C38B
:100DC90095628563F0A4FFAEF0E5648E048F05FF9C
:100DD90012602CEDF4042561F56022E562D395617A
:100DE900401DE562C395618563F0A4FFAEF0E5643B
:100DF9008E048F05FF12602CED2561F560801DE5DD
:100E090061C395628563F0A4FFAEF0E5648E048F3B
:100E190005FF12602CEDF4042561F5602290006B4A
:100E2900E0B40170E54275F00A84FF7E008F60E549
:100E39004275F00A84ADF07C008D6375680A7535DA
:100E490005753624E560C394115005120D6A8006B4
:100E590090059AE0F560E56090005BF0E54275F079
:100E69000A84FF7E008F60E54275F00A84ADF07C4C
:100E7900008D6375680A75350575365AE560C39442
:100E8900115005120D6A80069005D0E0F560E56005
:100E990090000AF02290006BE0B4016AE54275F017
:100EA9000A84FF7E008F60E54275F00A84ADF07C0C
:100EB900008D6375680A753505753636E560C39426
:100EC900115005120D6A80069005ACE0F560856049
:100ED90074E54275F00A84FF7E008F60E54275F083
:100EE9000A84ADF07C008D6375680A753505753621
:100EF90048E560C394115005120D6A80069005BE3D
:100F0900E0F56085607522E53A75F00484FF7E009E
:100F19008F60E53A75F00484ADF07C008D637568E7
:100F290004753501753600E560C3943F5005120D0F
:100F39006A80069001A4E0F56085605275510090C1
:100F49000031E075F020A4FFAEF09000B6E08E0409
:100F59008F05FF12602C8D6090009EE0D3953A506A
:100F6900030210169000C2E0D3953A4010ED9001AB
:100F7900A512606EE0F55475530002101390008DB0
:100F8900E0D3953A4043E5609001A512606EE0F523
:100F990061E5609001C512606EE0F5629000C2E003
:100FA900F404253AF56390008DE0FE9000C2E0F468
:100FB900042EF564E561B562058561608003120D53
:100FC900E48560547553008041E5609001C5126065
:100FD9006EE0F561E5609001E512606EE0F5629002
:100FE900008DE0F404253AF56390009EE0FE900040
:100FF9008DE0F4042EF564E561B5620585616080D4
:1010090003120DE48560547553000210BD9000C5AC
:10101900E0D3953A5011E56090022512606EE0F533
:10102900547553000210BD90008EE0D3953A504399
:10103900E56090020512606EE0F561E560900225B9
:1010490012606EE0F56290008EE0F404253AF563D3
:101059009000C5E0FE90008EE0F4042EF564E56191
:10106900B562058561608003120DE485605475538E
:10107900008041E5609001E512606EE0F561E56090
:1010890090020512606EE0F56290009EE0F404257E
:101099003AF56390008EE0FE90009EE0F4042EF590
:1010A90064E561B562058561608003120DE48560C0
:1010B90054755300229000D6E0F5657568117535B1
:1010C90002753600AE29AF2AE56575F00FA4FDACAF
:1010D900F0EDD39FEC9E4021E5658E048F05FF124C
:1010E900602CED75F010A4FFAEF0E53A75F01184AF
:1010F900FD7C00ED2FF566800EE53A75F01184FF51
:101109007E00EF24F0F566856660E53A75F0118496
:10111900AFF07E008F63120D6A856067AE29AF2A32
:101129009000D6E075F00FA4FDACF0EDD39FEC9ED6
:101139004028753502753610856660120D6A856717
:1011490061856062AE29AF2AE5658E048F05FF12BD
:1011590060578D63856564120DE485605275510091
:10116900755464755300229000D6E0F565756811D1
:10117900753502753600AE29AF2AE56575F00FA4FD
:10118900FDACF0EDD39FEC9E4021E5658E048F0503
:10119900FF12602CED75F010A4FFAEF0E53C75F080
:1011A9001184FD7C00ED2FF566800EE53C75F0118C
:1011B90084FF7E00EF24F0F566856660E53C75F0F6
:1011C9001184AFF07E008F63120D6A856067AE29C6
:1011D900AF2A9000D6E075F00FA4FDACF0EDD39FD7
:1011E900EC9E4028753502753610856660120D6AC9
:1011F900856761856062AE29AF2AE5658E048F0532
:10120900FF1260578D63856564120DE48560527520
:101219005100E5466017E546C394FE50109000CA98
:10122900E0B402099000B8E0D3940B50028017AEE5
:1012390051AF52E54612603C74E78E048F05FF12E8
:10124900602C8C518D529000A0E0B40453E53A759E
:10125900F00484FF7E008F60E53A75F00484ADF0F8
:101269007C008D63756804753501753600E560C3CA
:10127900943F5005120D6A80069001A4E0F560AE16
:1012890051AF52E56012603C74648E048F05FF1201
:10129900602CAE51AF52EF2DFDEE3CFC8C518D52BE
:1012A9007554647553002290006BE0B40146E54221
:1012B90075F00A84FF7E008F60E54275F00A84ADFF
:1012C900F07C008D6375680A753505753600E56033
:1012D900C394115005120D6A8006900576E0F560F9
:1012E900AE53AF54E5602FFF50010E746412608055
:1012F9008E538F5490006CE0B40146E54375F00AB3
:1013090084FF7E008F60E54375F00A84ADF07C00B0
:101319008D6375680A75350575366CE560C394117A
:101329005005120D6A80069005E2E0F560AE53AFF4
:1013390054E5602FFF50010E74641260808E538F44
:101349005490007BE0B40249E545C3944175F0052A
:1013590084FF7E008F60E54575F00584ADF07C0063
:101369008D63756805753506753600E560C3941398
:101379005005120D6A8006900678E0F560AE53AF0D
:1013890054E5602FFF50010E74641260808E538FF4
:10139900549000BDE0B40202800302144FE53A758F
:1013A900F01584FF7E008F60E53A75F01584ADF085
:1013B9007C008D637568157535037536F4E560C372
:1013C900940B5005120D6A8006900464E0F560E5FF
:1013D9006075F0FFA4FFAEF09000BEE08E048F05AB
:1013E900FF12602CED900054F0E54175F078A4FFF0
:1013F900AEF074FF8E048F05FF12602C8C358D368C
:1014090074028C068D071200398F60AC35AD3674C5
:1014190004FF1260578D63756804753506753628A3
:10142900E560C3941D5005120D6A80069006AAE076
:10143900F560AE53AF54E5602FFF50010E7464128E
:1014490060808E538F5490006AE0B4025DE53C756C
:10145900F064A4FFAEF074081200398E378F387427
:10146900058E048F05FF12602C8D60AE37AF38747E
:10147900058E048F05FF1260578D637568057535F4
:10148900057536DEE560C394135005120D6A8006B2
:10149900900656E0F560AE53AF54E5602FFF50015A
:1014A9000E74641260808E538F549000ACE0703CCF
:1014B900900031E075F00584FF7E008F6090003167
:1014C900E075F00584ADF07C008D637568057535B0
:1014D900057536C0E560C3941D5005120D6A800676
:1014E900900642E0F560E56090005CF022900073A0
:1014F900E0B401179007B0E02554FFAE5350010E38
:101509009000C7E01260808E538F549000EBE0B4D6
:1015190001149000ECE0A829B80004952A5007E5C9
:101529003AC3953B40028012900095E02554FFAEE6
:101539005350010E8E538F54802F900073E0B403E3
:1015490016A229B3B350109007B3E0C39405A82994
:10155900B80006952A40028010900095E02554FFB6
:10156900AE5350010E8E538F5490006DE0B40202B9
:1015790080030218F4900070E0602FE542D394468E
:10158900402890000BE0FEA3E0FF9000ABE075F06F
:1015990003A4FDACF0EFD39DEE9C400E9000CFE08C
:1015A900A829B80005D3952A50030218F49000A081
:1015B900E0B403028003021758853C367535009064
:1015C9000077E0A829B80004952A500E900078E029
:1015D900A835B80005D395365003021755E53C7573
:1015E900F002A4FFAEF074158E048F05FF12602C73
:1015F9008C068D079005F5126063FEE0FFEE900002
:101609006FE0FEEF8E0088F0A4FFAEF074648E04E4
:101619008F05FF12602C8C358D36900031E075F006
:1016290018A4FFAEF09000B6E08E048F05FF12609B
:101639002C8C068D0790060D126063AE35AF36E02F
:1016490012603C74648E048F05FF12602C8C358DFA
:1016590036E540A835B80077D395364072E540C3E2
:101669009536FFE49535FE8E358F367428BE000316
:101679009F500C753628753500740D900032F0AE08
:1016890035AF36900070E012603C74288E048F05E7
:10169900FF12602C8C358D36AE51AF52740A8E0410
:1016A9008F05FF12602C8D068C07AC35AD36CFCE79
:1016B900CF120003740A8E048F05FF12602C8C353B
:1016C9008D36AE51AF521260888E518F52807DE5B2
:1016D90040A835B8000495365072AE35AF36E540AE
:1016E9001260808E358F367428BE00039F500C75AA
:1016F9003628753500740D900032F0AE35AF36904E
:101709000070E012603C74288E048F05FF12602C73
:101719008C358D36AE51AF52740A8E048F05FF1287
:10172900602C8D068C07AC35AD36CFCECF120003B9
:10173900740A8E048F05FF12602C8C358D36AE51DC
:10174900AF52EF2DFDEE3CFC8C518D520218F490F6
:1017590000B8E0853AF0A4FFAEF0740512603C745D
:10176900071200398E358F36900077E0A829B80026
:1017790004952A5012900078E075F002A4FDACF0AF
:10178900EFC39DEE9C40030218F4E53A75F00B8413
:10179900FF7E009005F5126063FEE0FFEE90006F9A
:1017A900E0FEEF8E0088F0A4FFAEF074648E048F23
:1017B90005FF12602C8C358D36900031E075F018DC
:1017C900A4FFAEF09000B6E08E048F05FF12602CE6
:1017D9008C068D0790060D126063AE35AF36E012A8
:1017E900603C74648E048F05FF12602C8C358D3635
:1017F900E540A835B80077D395364072E540C395E2
:1018090036FFE49535FE8E358F367428BE00039F6A
:10181900500C753628753500740D900032F0AE35D0
:10182900AF36900070E012603C74288E048F05FF7B
:1018390012602C8C358D36AE51AF52740A8E048FDE
:1018490005FF12602C8D068C07AC35AD36CFCECF97
:10185900120003740A8E048F05FF12602C8C358DDB
:1018690036AE51AF521260888E518F52807DE5405D
:10187900A835B8000495365072AE35AF36E540123A
:1018890060808E358F367428BE00039F500C7536E4
:1018990028753500740D900032F0AE35AF369000E2
:1018A90070E012603C74288E048F05FF12602C8C46
:1018B900358D36AE51AF52740A8E048F05FF126012
:1018C9002C8D068C07AC35AD36CFCECF1200037404
:1018D9000A8E048F05FF12602C8C358D36AE51AF00
:1018E90052EF2DFDEE3CFC8C518D52229000CBE045
:1018F900B4026AE53A75F00884FF7E008F60E53A24
:1019090075F00884ADF07C008D6375680875350144
:101919007536E0E560C3943F5005120D6A80069064
:101929000264E0F560856056755500AE55AF56AC5A
:1019390053AD5412000374648E048F05FF12602C9A
:101949008C558D56900068E08C068D0712603C74AA
:10195900648E048F05FF12602C8C558D56AE51AFE5
:1019690052AC53AD5412000374648E048F05FF12F8
:10197900602C8C518D52900068E08C068D071260A6
:101989003C74648E048F05FF12602C8C518D52A219
:101999000D401DAE29AF2A7405BE00039F5002D227
:1019A9000DE53CD394CC4008D2017411900032F07B
:1019B9009000CAE0B402089000B8E0640B600280AD
:1019C90035AE51AF52E54612603C74E78E048F057F
:1019D900FF12602C8C518D529000CBE0B40217AEEF
:1019E90055AF56E54612603C74E78E048F05FF1229
:1019F900602C8C558D5690008AE05402601B900033
:101A090081E0A829B80012D3952A400DA20DB3B3DD
:101A19005007E53CC3949A40028028AE5DAF5E90C2
:101A2900007FE075F002A4FDACF0EF2DFDEE3CFC6B
:101A390074022DFD50010CE53CBC0007D39D400309
:101A4900756C01853C5E755D00E56C7003021B38A1
:101A59009000DDE0C3956C5003021B2A9000EDE075
:101A6900C394025076E54275F00A84FF7E00900522
:101A790065126063E0F536753500AE35AF36900016
:101A890080E012603C74648E048F05FF12602C8C18
:101A9900378D389000DDE004C3956C8C068D0712F4
:101AA900603C9000DDE08E048F05FF12602C8C37BE
:101AB9008D38AE51AF52EF2DFDEE3CFC8C518D525D
:101AC9009000CBE0B40212AE55AF56AA37AB38EF4F
:101AD9002BFBEE3AFA8A558B5680469000DDE004DE
:101AE900C3956C8574F0A4FFAEF09000DDE08E0420
:101AF9008F05FF12602C8C378D38AE51AF52EF2D08
:101B0900FDEE3CFC8C518D529000CBE0B40212AE3C
:101B190055AF56AA37AB38EF2BFBEE3AFA8A558BFD
:101B290056056C9000DDE0C3956C5003756C009010
:101B3900008AE05401601B90007EE0A829B80012D9
:101B4900D3952A400DA20DB3B35007E53AC394CCFF
:101B59004002802590007CE075F003A4FFAEF0E51B
:101B6900692FFF50010E74032FFF50010EE53ABE95
:101B79000007D39F4003756D01853A69E56D7003D0
:101B8900021C6B9000DEE0C3956D5003021C5D9052
:101B990000EDE0C394025076E54275F00A84FF7EB9
:101BA90000900565126063E0F536753500AE35AF16
:101BB9003690007DE012603C74648E048F05FF123C
:101BC900602C8C378D389000DEE004C3956D8C064F
:101BD9008D0712603C9000DEE08E048F05FF1260D5
:101BE9002C8C378D38AE51AF52EF2DFDEE3CFC8C6D
:101BF900518D529000CBE0B40212AE55AF56AA37C0
:101C0900AB38EF2BFBEE3AFA8A558B56804690009B
:101C1900DEE004C3956D8575F0A4FFAEF09000DE9B
:101C2900E08E048F05FF12602C8C378D38AE51AFD2
:101C390052EF2DFDEE3CFC8C518D529000CBE0B45F
:101C49000212AE55AF56AA37AB38EF2BFBEE3AFA74
:101C59008A558B56056D9000DEE0C3956D5003756E
:101C69006D009000E0E02552FFAE5150010E8E51FB
:101C79008F5290008FE0A851B800049552500990F6
:101C8900008FE0F5527551009000CBE0B4020D9041
:101C9900008FE0A855B800069556400280099000CB
:101CA9008FE0F556755500229000CBE0B401028013
:101CB90003021DBCA20DB35003021DBA900096E0A9
:101CC900B40168AE51AF52AC29AD2A120003743C7D
:101CD9008E048F05FF12602C9000A6E0BC00109DB9
:101CE900400D9000A8E0A851B8000495525002D2C6
:101CF90002AE51AF52AC29AD2A120003743C8E04D6
:101D09008F05FF12602C9000A6E0C3940ABC001551
:101D1900D39D40119000A8E0C39405A851B80005CF
:101D2900D3955250028002C2028068AE51AF52ACC4
:101D390029AD2A12000374788E048F05FF12602CD6
:101D49009000A6E0BC00109D400D9000A8E0A851AD
:101D5900B8000495525004D2028038AE51AF52AC4B
:101D690029AD2A12000374788E048F05FF12602CA6
:101D79009000A6E0C3940ABC0015D39D40119000C1
:101D8900A8E0C39405A851B80005D3955250028024
:101D990002C202A202B34019AE51AF529000A7E0AD
:101DA90012603C74648E048F05FF12602C8C518D77
:101DB900528002C202A200B34006A201B3B3500985
:101DC900900011E4F0A3F08024AE51AF527400D317
:101DD9009F74019E400C900011E551F0A3E552F06B
:101DE900800B74FF900011F8E4F0E8A3F09000ADC7
:101DF900E0D39402400C900098E07006A20DB3B3B2
:101E09004002801AAE51AF52740212603C8E518F5B
:101E190052AE55AF56740212603C8E558F569000E3
:101E290096E0B4011AAE51AF52740212603C8E5161
:101E39008F52AE55AF56740212603C8E558F56AE16
:101E490051AF52745E12603C740A8E048F05FF1202
:101E5900602C8C518D529000CBE0B40217AE55AF77
:101E690056745E12603C740A8E048F05FF12602C52
:101E79008C558D56AE51AF527402BE000AD39F40A5
:101E890006755202755100AE55AF567402BE000A6E
:101E9900D39F400675560275550090000FE551F025
:101EA900A3E552F022900031E090036512606EE0E4
:101EB900F56A756B64900031E0FE9000A1E0D39E55
:101EC9004037E53A75F00884FF7E008F60E53A7582
:101ED900F00884ADF07C008D63756808753503756D
:101EE9003696E560C3941F5005120D6A800690046A
:101EF9001AE0F56085606B8035E53A75F00884FF76
:101F09007E008F60E53A75F00884ADF07C008D6342
:101F19007568087535037536B6E560C3941F5005B5
:101F2900120D6A800690043AE0F56085606B229094
:101F390000D7E0F565756811753504753600AE2969
:101F4900AF2AE56575F00FA4FDACF0EDD39FEC9ECB
:101F59004021E5658E048F05FF12602CED75F010A8
:101F6900A4FFAEF0E53A75F01184FD7C00ED2FF584
:101F790066800EE53A75F01184FF7E00EF24F0F5D6
:101F890066856660E53A75F01184AFF07E008F636F
:101F9900120D6A856067AE29AF2A9000D7E075F007
:101FA9000FA4FDACF0EDD39FEC9E40287535047568
:101FB9003610856660120D6A856761856062AE2993
:101FC900AF2AE5658E048F05FF1260578D6385651D
:101FD90064120DE485606A756B64229000D7E0F5A0
:101FE90065756811753504753600AE29AF2AE56542
:101FF90075F00FA4FDACF0EDD39FEC9E4021E56593
:102009008E048F05FF12602CED75F010A4FFAEF061
:10201900E53C75F01184FD7C00ED2FF566800EE539
:102029003C75F01184FF7E00EF24F0F5668566604B
:10203900E53C75F01184AFF07E008F63120D6A855F
:102049006067AE29AF2A9000D7E075F00FA4FDAC08
:10205900F0EDD39FEC9E40287535047536108566E2
:1020690060120D6A856761856062AE29AF2AE565F0
:102079008E048F05FF1260578D63856564120DE428
:1020890085606A756B649000A0E0B40479900031B2
:10209900E0FE9000A1E0D39E4037E53A75F0088450
:1020A900FF7E008F60E53A75F00884ADF07C008D05
:1020B90063756808753503753696E560C3941F50D6
:1020C90005120D6A800690041AE0F56085606B8040
:1020D90035E53A75F00884FF7E008F60E53A75F0C2
:1020E9000884ADF07C008D63756808753503753615
:1020F900B6E560C3941F5005120D6A800690043A34
:10210900E0F56085606B2290006BE0B4013BE5422D
:1021190075F00A84FF7E008F60E54275F00A84AD90
:10212900F07C008D6375680A753505753612E560B2
:10213900C394115005120D6A8006900588E0F56078
:10214900E56B2560C39464F56B90006CE0B4013BCA
:10215900E54375F00A84FF7E008F60E54375F00A58
:1021690084ADF07C008D6375680A75350575367E1A
:10217900E560C394115005120D6A80069005F4E0DC
:10218900F560E56B2560C39464F56BE56A256BF52D
:102199005F900073E0B402109007AFE0255FFE90F6
:1021A90000C7E0F4042EF55F9000CAE0D394014023
:1021B90040E546C394E7501D74E7C39546FE900772
:1021C900B1E08E00F5F0E884FF7E008F60E55F25C1
:1021D90060F55F801CE546C394E7FE9007B1E08E89
:1021E90000F5F0E884FF7E008F60E55FC39560F538
:1021F9005FA20D4006E56A2464F55FE55FD3946448
:102209004009E55FC39464F55F8003755F00900042
:10221900A3E0C3955F50069000A3E0F55F22D200CA
:1022290090005AE0A829B80004952A504190005A14
:10223900E0A829B80004952A5003755F0F90005A49
:10224900E004A829B80004952A5003755F0A900094
:102259005AE02402A829B80004952A5005755F059B
:10226900C20090005AE060067409900032F0C23949
:102279007E017F009000A9E012603C9000B8E08EDA
:10228900048F05FF12602CE53ABC0017D39D40135B
:102299009000B2E0B40204D2398002C200740A90FC
:1022A9000032F09000AAE0C3954250159000BCE0BE
:1022B900A829B80004952A5002C200740B90003274
:1022C900F0E542C39464501D900102E0600D900155
:1022D90002E0A829B80006952A40028008C20074C5
:1022E9000B900032F0A2004003755F059000EBE00F
:1022F900B401149000ECE0A829B80004952A50070D
:10230900E53AC3953B40028008900094E0F55F8070
:102319003A900073E0B40306A229B3B34002802BBC
:102329009007B3E0C39405A829B80004952A500C76
:10233900900094E0F55F740C900032F09007B3E0E0
:10234900A829B80004952A5002C200855F47900069
:1023590065E0255FFE900031E075F01E84FC7F008A
:10236900EE2CF55F22900031E075F00584FF7E00C8
:102379008F60900031E075F00584ADF07C008D63CD
:102389007568057535037536D69000B6E01475F095
:102399000584FF7E00E560BE00039F5005120D6AAB
:1023A900800BE56090043B12606EE0F560E560909B
:1023B90007B2F09007B2E0FE9000A5E0C39E500876
:1023C9009000A5E09007B2F022E54275F00A84FF7B
:1023D9007E00900565126063E0F56FE56FD3946444
:1023E9004010E56FC3946475F00F84FF7E008F6F12
:1023F9008003756F00900088E0256FF56F229000CB
:10240900A0E0C39403502690079FE0FEA3E0FF7469
:1024190004120039E53A12603C740F8E048F05FFEF
:1024290012602C90079DECF0A3EDF0802490079F9B
:10243900E0FEA3E0FF7404120039E53C12603C742D
:102449000F8E048F05FF12602C90079DECF0A3ED11
:10245900F090007BE0B40262E545C3944175F00554
:1024690084FF7E008F60E54575F00584ADF07C0042
:102479008D63756805753506753614E560C394175F
:102489005005120D6A800690068CE0F56090079D54
:10249900E0FEA3E0FF740A8E048F05FF12602CE5AD
:1024A900608C068D0712603C740A8E048F05FF123A
:1024B900602C90079DECF0A3EDF090079DE0FEA342
:1024C900E0FF9007A3E0FCA3E0FDEDD39FEC9E4065
:1024D9000F9007A3E0F8A3E090079DC8F0A3C8F008
:1024E900229006ACE090386BF8282873804C852A36
:1024F9004F80479000B8E0853AF0A4FFAEF0740829
:102509001200398F4F8033853C4F802E85424F8092
:102519002985434F802485444F801F85454F801A64
:1025290085464F801585414F801085404F800B852A
:0A253900474F8006900012E0F54FB6
:10386B000224F50224F70224FC022510022515027E
:10387B00251A02251F02252402252902252E0225A1
:07388B003302253802253D40
:102543009006ADE0FE9006AEE0D39E404B9006AC05
:10255300E0B404189006AEE0C3954F5002D22A901F
:1025630006ADE0D3954F4002C22A802A9006ADE023
:10257300C3954F50099006AEE0D3954F50028002A9
:10258300D22A9006ADE0D3954F50099006AEE0C332
:10259300954F5002C22A802A9006ADE0D3954F4052
:1025A300099006AEE0C3954F40028002C22A90060E
:1025B300ADE0C3954F40099006AEE0D3954F40027E
:1025C300D22A229006B0E0903892F8282873804CE3
:1025D300852A4F80479000B8E0853AF0A4FFAEF01B
:1025E30074081200398F4F8033853C4F802E85420B
:1025F3004F802985434F802485444F801F85454F55
:10260300801A85464F801585414F801085404F8045
:0C2613000B85474F8006900012E0F54F49
:103892000225D10225D30225D80225EC0225F10208
:1038A20025F60225FB02260002260502260A02262A
:0738B2000F02261402261983
:10261F009006B1E0FE9006B2E0D39E405F9006B008
:10262F00E0B404189006B2E0C3954F5002D22B903D
:10263F0006B1E0D3954F4002C22B803E9006B1E029
:10264F00C3954F50099006B2E0D3954F50028002C8
:10265F00D22B9006B1E0D3954F50099006B2E0C34C
:10266F00954F5002C22B9006B0E0B401099000C400
:10267F00E0D3953C50028002C22B802A9006B1E035
:10268F00D3954F40099006B2E0C3954F40028002A8
:10269F00C22B9006B1E0C3954F40099006B2E0D32C
:1026AF00954F4002D22B229006B4E09038B9F8280B
:1026BF002873804C852A4F80479000B8E0853AF008
:1026CF00A4FFAEF074081200398F4F8033853C4F52
:1026DF00802E85424F802985434F802485444F802B
:1026EF001F85454F801A85464F801585414F8010B5
:1026FF0085404F800B85474F8006900012E0F54FC5
:1038B9000226C10226C30226C80226DC0226E1022C
:1038C90026E60226EB0226F00226F50226FA022651
:0738D900FF0227040227098A
:10270F009006B5E0FE9006B6E0D39E404B9006B41F
:10271F00E0B404189006B6E0C3954F5002D22C9047
:10272F0006B5E0D3954F4002C22C802A9006B5E043
:10273F00C3954F50099006B6E0D3954F50028002D3
:10274F00D22C9006B5E0D3954F50099006B6E0C352
:10275F00954F5002C22C802A9006B5E0D3954F407A
:10276F00099006B6E0C3954F40028002C22C900636
:10277F00B5E0C3954F40099006B6E0D3954F4002A0
:10278F00D22C229006B8E09038E0F8282873804CBD
:10279F00852A4F80479000B8E0853AF0A4FFAEF04D
:1027AF0074081200398F4F8033853C4F802E85423D
:1027BF004F802985434F802485444F801F85454F87
:1027CF00801A85464F801585414F801085404F8078
:0C27DF000B85474F8006900012E0F54F7C
:1038E00002279D02279F0227A40227B80227BD02B4
:1038F00027C20227C70227CC0227D10227D60227D8
:07390000DB0227E00227E5CE
:1027EB009006B9E0FE9006BAE0D39E404B9006B837
:1027FB00E0B404189006BAE0C3954F5002D22D9066
:10280B0006B9E0D3954F4002C22D802A9006B9E05D
:10281B00C3954F50099006BAE0D3954F50028002F2
:10282B00D22D9006B9E0D3954F50099006BAE0C36C
:10283B00954F5002C22D802A9006B9E0D3954F4098
:10284B00099006BAE0C3954F40028002C22D900654
:10285B00B9E0C3954F40099006BAE0D3954F4002BB
:10286B00D22D229006BCE0903907F8282873804CB3
:10287B00852A4F80479000B8E0853AF0A4FFAEF070
:10288B0074081200398F4F8033853C4F802E854260
:10289B004F802985434F802485444F801F85454FAA
:1028AB00801A85464F801585414F801085404F809B
:0C28BB000B85474F8006900012E0F54F9F
:1039070002287902287B022880022894022899023B
:10391700289E0228A30228A80228AD0228B202285E
:07392700B70228BC0228C111
:1028C7009006BDE0FE9006BEE0D39E404B9006BC4E
:1028D700E0B404189006BEE0C3954F5002D22E9084
:1028E70006BDE0D3954F4002C22E802A9006BDE078
:1028F700C3954F50099006BEE0D3954F5002800212
:10290700D22E9006BDE0D3954F50099006BEE0C386
:10291700954F5002C22E802A9006BDE0D3954F40B6
:10292700099006BEE0C3954F40028002C22E900672
:10293700BDE0C3954F40099006BEE0D3954F4002D6
:10294700D22E229006C0E090392EF8282873804CAA
:10295700852A4F80479000B8E0853AF0A4FFAEF093
:1029670074081200398F4F8033853C4F802E854283
:102977004F802985434F802485444F801F85454FCD
:10298700801A85464F801585414F801085404F80BE
:0C2997000B85474F8006900012E0F54FC2
:10392E0002295502295702295C02297002297502C3
:10393E00297A02297F02298402298902298E0229E5
:07394E009302299802299D54
:1029A3009006C1E0FE9006C2E0D39E404B9006C065
:1029B300E0B404189006C2E0C3954F5002D22F90A2
:1029C30006C1E0D3954F4002C22F802A9006C1E092
:1029D300C3954F50099006C2E0D3954F5002800231
:1029E300D22F9006C1E0D3954F50099006C2E0C3A1
:1029F300954F5002C22F802A9006C1E0D3954F40D5
:102A0300099006C2E0C3954F40028002C22F900690
:102A1300C1E0C3954F40099006C2E0D3954F4002F1
:102A2300D22F229006C4E0903955F8282873804CA1
:102A3300852A4F80479000B8E0853AF0A4FFAEF0B6
:102A430074081200398F4F8033853C4F802E8542A6
:102A53004F802985434F802485444F801F85454FF0
:102A6300801A85464F801585414F801085404F80E1
:0C2A73000B85474F8006900012E0F54FE5
:10395500022A31022A33022A38022A4C022A51024B
:103965002A56022A5B022A60022A65022A6A022A6C
:073975006F022A74022A7997
:102A7F009006C5E0FE9006C6E0D39E404B9006C47C
:102A8F00E0B404189006C6E0C3954F5002D23090C0
:102A9F0006C5E0D3954F4002C230802A9006C5E0AC
:102AAF00C3954F50099006C6E0D3954F5002800250
:102ABF00D2309006C5E0D3954F50099006C6E0C3BB
:102ACF00954F5002C230802A9006C5E0D3954F40F3
:102ADF00099006C6E0C3954F40028002C2309006AF
:102AEF00C5E0C3954F40099006C6E0D3954F40020D
:102AFF00D230229006C8E090397CF8282873804C99
:102B0F00852A4F80479000B8E0853AF0A4FFAEF0D9
:102B1F0074081200398F4F8033853C4F802E8542C9
:102B2F004F802985434F802485444F801F85454F13
:102B3F00801A85464F801585414F801085404F8004
:0C2B4F000B85474F8006900012E0F54F08
:10397C00022B0D022B0F022B14022B28022B2D02D3
:10398C002B32022B37022B3C022B41022B46022BF3
:07399C004B022B50022B55DA
:102B5B009006C9E0FE9006CAE0D39E404B9006C893
:102B6B00E0B404189006CAE0C3954F5002D23190DE
:102B7B0006C9E0D3954F4002C231802A9006C9E0C6
:102B8B00C3954F50099006CAE0D3954F500280026F
:102B9B00D2319006C9E0D3954F50099006CAE0C3D5
:102BAB00954F5002C231802A9006C9E0D3954F4011
:102BBB00099006CAE0C3954F40028002C2319006CD
:102BCB00C9E0C3954F40099006CAE0D3954F400228
:102BDB00D231229006CCE09039A3F8282873804C90
:102BEB00852A4F80479000B8E0853AF0A4FFAEF0FD
:102BFB0074081200398F4F8033853C4F802E8542ED
:102C0B004F802985434F802485444F801F85454F36
:102C1B00801A85464F801585414F801085404F8027
:0C2C2B000B85474F8006900012E0F54F2B
:1039A300022BE9022BEB022BF0022C04022C09025E
:1039B3002C0E022C13022C18022C1D022C22022C7A
:0739C30027022C2C022C311D
:102C37009006CDE0FE9006CEE0D39E404B9006CCAA
:102C4700E0B404189006CEE0C3954F5002D23290FC
:102C570006CDE0D3954F4002C232802A9006CDE0E0
:102C6700C3954F50099006CEE0D3954F500280028E
:102C7700D2329006CDE0D3954F50099006CEE0C3EF
:102C8700954F5002C232802A9006CDE0D3954F402F
:102C9700099006CEE0C3954F40028002C2329006EB
:102CA700CDE0C3954F40099006CEE0D3954F400243
:102CB700D232229006D0E09039CAF8282873804C87
:102CC700852A4F80479000B8E0853AF0A4FFAEF020
:102CD70074081200398F4F8033853C4F802E854210
:102CE7004F802985434F802485444F801F85454F5A
:102CF700801A85464F801585414F801085404F804B
:0C2D07000B85474F8006900012E0F54F4E
:1039CA00022CC5022CC7022CCC022CE0022CE502E8
:1039DA002CEA022CEF022CF4022CF9022CFE022D06
:0739EA0003022D08022D0D60
:102D13009006D1E0FE9006D2E0D39E404B9006D0C1
:102D2300E0B404189006D2E0C3954F5002D233901A
:102D330006D1E0D3954F4002C233802A9006D1E0FA
:102D4300C3954F50099006D2E0D3954F50028002AD
:102D5300D2339006D1E0D3954F50099006D2E0C309
:102D6300954F5002C233802A9006D1E0D3954F404D
:102D7300099006D2E0C3954F40028002C233900609
:102D8300D1E0C3954F40099006D2E0D3954F40025E
:102D9300D23322AE57AF5874F5D39F74019E4008C7
:102DA3007857126090022EB0755801755700AE29FE
:102DB300AF2AE56FBE000DD39F400990009AE0D380
:102DC300957040028023757000E56FC3952AF54F17
:102DD30090009DE0D3956E4008E56E254FF56E801B
:102DE3000690009DE0F56E80020570900076E0D3BA
:102DF300953C401CE53AC3953B4015AE29AF2AE507
:102E03006FBE00039F500990009BE0D39571400271
:102E1300806E9007B6E0A829B80004952A50037580
:102E230073009007B6E0A829B8000BD3952A400693
:102E3300E52A9007B6F0E5737041E52AC3956FF56F
:102E43004FE54FD394054003754F0590009CE0C3B5
:102E5300956E5007E54FC3956E40028009E56EC33A
:102E6300954FF56E800690009CE0F56E90009CE017
:102E7300D3956E400690009CE0F56E75710080025C
:102E83000571E5737016900076E0C3953C500DE52F
:102E93006F2405A829B80006952A4002800F9000E8
:102EA30089E0F56E75730174789007B6F022AE571A
:102EB300AF5874E9D39F74039E400878571260900B
:102EC30002304F755801755700756E32A234402A8F
:102ED300756E19900089E075F002A4FFAEF0E570FD
:102EE300BE0006D39F4002D2340570757303747815
:102EF3009007B6F075720002303EAE29AF2AE56F37
:102F03006F4E700302303EE56FBE000DD39F400944
:102F130090009AE0D395704002800F757000E573BE
:102F2300C394035003756E19800DE56FC3952AF59D
:102F33004FE570254FF570900076E0D3953C400E39
:102F43009007B6E0A829B80007D3952A4002800C61
:102F53000572900089E0B57203757300E573B403DD
:102F630006A20DB3B34002800A0572E572B43C03B6
:102F7300757302E573B402299007B6E0A829B80077
:102F83000ED3952A4009E52A9007B6F07572009092
:102F93000076E0C3953C500975720074789007B6CB
:102FA300F0E573705A900076E0D3953C401CE53A07
:102FB300C3953B4015AE29AF2AE56FBE00039F5072
:102FC3000990009BE0D395714002800875710075EC
:102FD3006E4B8028E52AC3956FF54FE54FD39405D3
:102FE3004003754F05900076E0D3953C4008E571AA
:102FF300254FF5718006E5712406F571757200E5BC
:10300300737016900076E0C3953C500DE56F240570
:10301300A829B80006952A40028003757301E57359
:10302300B40118756E190572900089E0B5720675C2
:10303300730275720074789007B6F0E56E75F00A46
:10304300A4FFAEF09007A7EEF0A3EFF022E54A90BD
:1030530039F1F828287390006EE0700302327790FC
:1030630000A4E0B401028003023192900030E0B585
:103073003902800302318F7E017F00E5BE12603C7E
:10308300E5BD2FFF50010E8E358F36741012603C54
:10309300900059E08E048F05FF12602C9007ABEC73
:1030A300F0A3EDF074FFBC00039D500B74FF900779
:1030B300ABF8E4F0E8A3F0E546600FE546C394FE01
:1030C30050089000CAE06402600280649000B8E097
:1030D300B40B1F9007ABE0FEA3E0FF74E712603C64
:1030E300E5468E048F05FF12602C9007ABECF0A32E
:1030F300EDF09000B8E0D3940B40089000A0E0649A
:10310300046002802B9007ABE0FEA3E0FF9007ADC5
:10311300E0FCA3E0FDEFD39DEE9C400D1260889090
:1031230007ABEEF0A3EFF080079007ABE4F0A3F05A
:1031330090006EE0B4021E9007ABE0FEA3E0FF90A8
:1031430007B7E02FFF50010E74011200399007AB4F
:10315300EEF0A3EFF09007ABE0FEA3E0FF9007B71C
:10316300E0BE0008D39F4004D2378002B2379007F5
:10317300ACE09007B7F09000A0E064016006A237CE
:10318300B3B3400280069007ACE0F53A023275D241
:10319300377E017F00E5BE12603CE5BD2FFF500185
:1031A3000E8E358F36741012603C900059E08E04F9
:1031B3008F05FF12602C9007ABECF0A3EDF0E54612
:1031C300600FE546C394FE50089000CAE0640260B5
:1031D3000280649000B8E0B40B1F9007ABE0FEA33D
:1031E300E0FF74E712603CE5468E048F05FF126032
:1031F3002C9007ABECF0A3EDF09000B8E0D3940B68
:1032030040089000A0E064046002802B9007ABE0CC
:10321300FEA3E0FF9007ADE0FCA3E0FDEFD39DEE3E
:103223009C400D1260889007ABEEF0A3EFF080078F
:103233009007ABE4F0A3F090006EE0B4021E900799
:10324300ABE0FEA3E0FF9007B7E02FFF50010E7441
:10325300011200399007ABEEF0A3EFF09007ACE05A
:103263009007B7F09000A0E0640160069007ACE01F
:10327300F53A8003753A0090006AE07006754A01DA
:1032830002305075BB1802384590006AE0700302A3
:1032930033FD7E017F00E5BE12603CE5BD2FFF508C
:1032A300010E8E358F369000B0E0B4010F7E0F7F94
:1032B300FFAC35AD361260888E358F369000D5E081
:1032C300B40245AE35AF3690001BE0FCA3E0FDED44
:1032D300D39FEC9E400A90001BE535F0A3E536F042
:1032E300AE35AF3690001DE0FCA3E0FDEFD39DEEBD
:1032F3009C400A90001DE535F0A3E536F0AE35AFEE
:103303003674041200398F3C9000D5E0704CAE3512
:10331300AF3690001BE0FCA3E0FDEFD39DEE9C4095
:10332300091260888E358F36800675360075350034
:10333300AE35AF36741012603C900056E08E048FA9
:1033430005FF12602C8C358D3674FFBC0009D39DAC
:10335300400585363C8003753CFE9000A0E0B40137
:103363000280030233FBA20DB3B3500E900074E04E
:10337300A829B80005D3952A500280719000B1E0C6
:10338300853CF0A4FFAEF074648E048F05FF1260D9
:103393002C8C358D36E5466016E546C394FE500FFA
:1033A3009000CAE0B402089000B8E0640B600280A9
:1033B30017AE35AF3674E712603CE5468E048F05D1
:1033C300FF12602C8C358D36AE35AF369007ABE0EF
:1033D300FCA3E0FDEDD39FEC9E400585363A800BC0
:1033E300A237B340069007ACE0F53A800BA237B39F
:1033F30040069007ACE0F53A8003753C0090006D01
:10340300E07006754A0202305075BB1902384590C8
:10341300006DE070030234B2E539D395284003020E
:1034230034B0900019E0FEA3E0FFE5401260809005
:103433000019EEF0A3EFF07E017F00E5BE12603CC1
:10344300E5BD2FFF50010E8E358F369000DAE07008
:1034530013740A12603C74518E048F05FF12602CA2
:103463008D408019AE35AF36740A12603C8F048EDE
:10347300057E017F95CDCCCD125F2A8F40E540D3E9
:1034830094644003754064900019E0FEA3E0FFE5F7
:10349300402FFF50010E900019EEF0A3EFF09000C3
:1034A30071E0048E048F05FF12602C8D408003753C
:1034B30040329000BDE07006754A0302305075BB80
:1034C300130238459000BDE0604A7E017F00E5BEEF
:1034D30012603CE5BD2FFF50010E8E358F3674040C
:1034E3001200398F419000BFE08541F0A4FDACF09C
:1034F3007464FF12602C8D419000BEE08541F0A4FE
:10350300FFAEF074FF8E048F05FF12602CED900068
:1035130055F0800375410090006BE07006754A0416
:1035230002305075BB1702384590006BE0B40102BE
:1035330080030235C07E017F00E5BE12603CE5BD1D
:103543002FFF50010E8E358F369007B8E06019902B
:1035530007B8E014905AB612008CE493FC740193FC
:10356300FDEDC39FEC9E400280069007B8E014F087
:103573009007B8E0C394B3501DAE35AF369007B88B
:10358300E004905AB612008CE493FC740193FDEFAF
:10359300C39DEE9C400280069007B8E004F09007BC
:1035A300B8E0FE900091E08E0088F0A4FFAEF074C6
:1035B300648E048F05FF12602C8D428003754200D8
:1035C30090006CE07006754A0502305075BB160218
:1035D300384590006CE0B4010280030236697E0135
:1035E3007F00E5BE12603CE5BD2FFF50010E8E3516
:1035F3008F369007B9E060199007B9E014905C200A
:1036030012008CE493FC740193FDEDC39FEC9E4088
:103613000280069007B9E014F09007B9E0C394B3B1
:10362300501DAE35AF369007B9E004905C20120010
:103633008CE493FC740193FDEFC39DEE9C400280E8
:10364300069007B9E004F09007B9E0FE900097E018
:103653008E0088F0A4FFAEF074648E048F05FF1211
:10366300602C8D43800375430075BB1F0238457E74
:10367300017F00E5BE12603CE5BD2FFF50010E8EB9
:10368300358F36740912603C74E68E048F05FF1281
:10369300602C8D45900073E07006754A0702305028
:1036A30075BB15023845900073E070030237C47E82
:1036B300017F00E5BE12603CE5BD2FFF50010E8E79
:1036C300358F3674041200398F44900073E0B401CF
:1036D300159000C7E08544F0A4FFAEF07407120014
:1036E30039EF9007B0F0900073E0B402159000C773
:1036F300E08544F0A4FFAEF07407120039EF9007A1
:10370300AFF0900073E0B4030280030237A7900088
:10371300B4E0701CE544C394195002D229E544D3A4
:1037230094644002C229900093E09007B3F0806351
:10373300900093E070349000C7E08544F0A4FFAE9E
:10374300F074FF8E048F05FF12602CED9007B3F029
:10375300AE29AF2A741EBE0006D39F4002D229E5CC
:103763003CD394E54002C2298029E544C3940A501E
:103773000DAE29AF2A741EBE0004D39F50028002EF
:10378300D229E53CD394E54002C229900093E0900E
:1037930007B3F09007B3E0C3940550067405900790
:1037A300B3F0C238900073E0B40414E544C3941931
:1037B3005002D238E544D394324002C238C2298041
:1037C300037544009000CAE07006754A0802305041
:1037D30075BB14806D9000CAE060567E017F00E5E2
:1037E300BE12603CE5BD2FFF50010E8E358F36EFC4
:1037F300D39421EE940E40057546FF8015AE35AF88
:1038030036741012603C74E38E048F05FF12602C33
:103813008D46E54675F00BA4FFAEF09000B8E08E40
:10382300048F05FF12602C9007ADECF0A3EDF08040
:103833000375460090006EE0600575BB1A80037542
:02384300BB18B0
:1039F10002305902328C0234120234C702352C02D1
:0B3A010035D50236720236A90237D814
:05384500054AD2EC224F
:09606E002582F58250020583220F
:0F008C0025E050020583258250020583F582226C
:10600B00EF2F500205832582F582E5833E2EF58323
:01601B002262
:10608000CFC39FFF50011E22C3EF9DFFEE9CFE2257
:086090000806B6000218062202
:0D604A00A3E004F07006120049E004F0220B
:0E003900048007C3CE13CECF13CFD5E0F6223E
:105F2A00BC000FBE0008ED8FF084FFADF022E4FE46
:105F3A00FF22BE000DEF60FE54F0606F20E70302FF
:105F4A005FE0EAC0E0EBC0E078017A0075F001EEAC
:105F5A0020E710EF25E0FFEE33FE0AC5F023C5F077
:105F6A0030E7F0EA5407F9096A7A007B0060010811
:105F7A00C3EC9E40167004ED9F4010ED9FFDEC9E11
:105F8A00FCE5F0CA4ACA03F5F08005E5F003F5F02E
:105F9A00C3EE13FEEF13FFD9D77908CACBCAD8D0FC
:105FAA00EAFEEBFFD0E0FBD0E0FA22EC8FF084FCB3
:105FBA00ED54F045F0C48FF084FEEDC454F045F082
:105FCA00C48FF084FDEEC4FE54F02DFFEE540F3C56
:105FDA00FEADF07C0022790078008FF0EC7E08207C
:105FEA00E70DC3CD33CD33C933C9C833C8DEF08416
:105FFA0049F9E5F08FF0BE00E6FD7C00E9FFE8FE16
:01600A002273
:0E603C00F88FF0A4FFE5F0CE88F0A42EFE222F
:10000300EF8DF0A4F9A8F0EF8CF0A428F8EE8DF0B2
:06001300A428FEE9FF2213
:10601C00600D782B026026007830D8FED5E0F8228F
:10602C00EEC0E07E00125F2AEFFDEEFCD0E0FE2217
:0C605700EEC0E07E00125F2AD0E0FE22C6
:03001B0002001EC2
:0300530002005652
:03009B00020071EF
:0300000002607724
:0960770075817A75D0000241F830
:0B606300E5822FF582E5833EF58322E5
:0A0049000582D5820215831582227C
:10001E00C0E0C0F0C083C082C0D075D0001241AD28
:0B002E00D0D0D082D083D0F0D0E032E0
:10005600C0E0C0F0C083C082C0D075D0001241B0ED
:10006600D0D0D082D083D0F0D0E032C0E0C0F0C093
:1000760083C082C0D075D0001241CFD0D0D082D0FC
:0600860083D0F0D0E0324F
:00000001FF
